:100000002500DF0C0200080C0600050C26006B0022
:100010006C006D0070007F00000C74096A004000E5
:10002000A909EA020F0A540A2C0CA909730909024A
:100030008C0043061E0A09022C00300AED03140A44
:10004000AF02290710050B02B0092700FF0C690653
:100050000702100707026F06070227006906320A27
:100060006D00140AE70473090902F80E2900480C10
:1000700089004306480A880C890043064A0A280C6E
:10008000890043064C0A180C890043064E0A6E0A82
:10009000010C590A020C590A030C590A040CEB0111
:1000A0001C0C8B0043066B000B02B0092700E70411
:1000B0006E0ACB01B0092E002E024306630A0E021F
:1000C0008909EE07660A73096906630A2E02430668
:1000D000710A0E02200D8909EE06710A730969067C
:1000E0006E0AE705140A0702280046044605080CB4
:1000F0002A0040006607010C9F006903680326047C
:1001000003062605A605A604EA02790A86058604E2
:1001100000082800E804080C2A0006040F0CA909AE
:10012000AF0928030306970A00000604990A06058A
:10013000990A0E0CA9090000EA02900AAF09AF095A
:1001400000000605200C2A004000A909EA02A40AC2
:1001500000083F00000000000000FF02AA0A00089B
:10016000E201920842084108C20887085008C40802
:10017000C3088C084E0848084908AB0845084A08D7
:100180004908A108D1084F080008C7084B084608CD
:0A0190004A088E084C08470848088A
:021FFE00EA0FE8
:00000001FF
